:0600000061C0FECFD9C073
:10000600FCCFFBCF91C0F9CFDAC0F7CFF6CFF5CF53
:10001600F4CFF3CF83C0F1CFF0CFEFCFEECFEDCF5C
:10002600ECCFEBCF1027E80364000A0001000010B4
:100036000001100001000000000024504D544B3315
:1000460031342C302C312C302C312C312C352C30B9
:100056002C302C302C302C302C302C302C302C30BA
:100066002C302C302C302C302A32430D0A002450F0
:100076004D544B3330312C302A32430D0A00245074
:100086004D544B3836392C312C302A33340D0A0076
:1000960024504D544B3235312C31343430302A32E1
:1000A600390D0A0024504D544B3232302C35303045
:1000B6002A32420D0A00040008003C000000F894B1
:1000C600EE27ECBBE5BFF8E1A895A4B7A77FA4BFD0
:1000D600F1BDE1BD8DE0A2E0ED938A95E9F780E8F8
:1000E600A0E6ED938A95E9F7ECEBF0E08591959122
:1000F600009761F0A591B59105901590BF01F001AB
:1001060005900D920197E1F7FB01F0CFE0E0E3BB2C
:10011600E4BBE5BBEFEDEDBFC0E872C1EA9398988A
:10012600E0E0E0BFE3BF49C0AA93EA93EFB7EA93E2
:1001360035D2A0E09999A1E0E1E0EA2711F4999877
:1001460001C0999A9F9B03C09F98E0E8EBBFC098B7
:10015600849B06C03394E5E0E31511F494983324A8
:10016600859B16C094982394E5E0E21589F4A0E0F7
:100176009A99A1E0E1E0EA2711F49A9801C09A9AC7
:100186002224E1E0E71520F0E71509F49B9A739421
:100196009B9B02C09C9901C007C05394E8E0E515FB
:1001A60019F49C9844245524E991EFBFE991A9914B
:1001B6001895EA939E9AE0E0EBBFE9911895EA93C9
:1001C600EFB7EA9345D21BB10CB1E12FEC7171F494
:1001D600E92D9394E0580083E8E0E91509F49924A1
:1001E600B394E8E0EB1511F4BB24A09A0991199198
:1001F600E991EFBFE99118951A93989AE2E0E0BF6A
:10020600E3E0E3BFE0E0E2BFE5EEE6BFE5E0E8BF3E
:10021600BB2011F4989901C001C0FACF989B0CC07D
:10022600E82D8394E0581081E8E0E81509F4882465
:10023600F894BA947894E12F19910895BA93AA93F1
:100246001A9310E0EB811E1750F4969AA981BA8191
:10025600F3D19698A981BA81EFD11F5FF3CF1881A8
:100266004AC1BA93AA93F4D100E010E0C498EB8196
:10027600F07099D1FE2FE0E08F01EA8194D1F0E091
:100286000E2B1F2BC49AF801E8D135C1AA93829987
:10029600FECFE881EFB9AAD1A9D1A8D1A7D1A6D11D
:1002A600A5D1A4D1A3D163C1A0E0BEEFDADFA6E950
:1002B600A2D1A8EDB0E8D5DFA0E2B6EAD2DFA5E08C
:1002C600B6ECCFDFA0EAB4E9CCDFACEEB2ECC9DF26
:1002D600A3E8BAECC6DFA6EDBEECC3DFABE9B4EC2F
:1002E600C0DFA5E5B8E9BDDFA7E7BCECBADFA0E053
:1002F600B0EEB7DFA0E0B8ECB4DFA0E0B0ECD3C05E
:10030600FF921A93E1E0FE2E10E0F0FE43C0239721
:1003160073DFEA83AA81A432B1F46EDFE9836CDF6E
:10032600E883A981A73419F4A881A03509F00BC088
:10033600F1FC0FC0E894F0F8E3E0EA93A4E6B0E03D
:100346007DDF239627C0123511F5EFE5E9B9A4E65E
:1003560052D1F894A0E4B0E00CD1A4E7B0E009D102
:10036600A4E8B0E006D1A6E9B0E003D1A4E643D103
:10037600EFE3E9B9A4EFB1E05FD1AAEAB0E0F9D0C2
:10038600E1E03BD1E894F1F810E0789401C01F5FFA
:100396002396BBCF1991FF900895E0E8E6BDE0E013
:1003A600E6BDE4E0EBBBE0E0EABBE5EDE7BBE4E19C
:1003B600E8BBE2E5E1BBEDE2E2BBE0E0EFBDE4E095
:1003C600EEBDECD0E0E0E5BDE4BDEBBDEABDE9BDC8
:1003D600E8BDE1E8E9BFE0E0E5BFE0E8EBBFEABF82
:1003E600E0E0EDB9EBB9E8E9EAB9E6E0E3B9E0E067
:1003F600E2B9EFE3E9B9E0E8E8B9E0E0E1B9089588
:10040600CCDF78947DDFF8944FDFE2E0F6D0789485
:10041600F8D0C29872D09899FDCF9B9B02C09C9B46
:1004260001C005C04394E6E0E41509F49C9ABB209C
:1004360029F09B9B02C09C9901C008C09E9B04C0EA
:10044600A1E073D09E989F9A30D0F1CFE1CFFFCF35
:10045600B39B23C0989AE2E0E0BFE3E0E3BFE0E0AD
:10046600E2BFE5EEE6BFE5E0E8BFB19902C09899C4
:1004760001C001C0FACFB39B02C0B19901C00DC043
:10048600C698C298C498B2D0B1D0B0D0AFD0AED0D2
:10049600ADD0ACD0ABD0EFB108950895A1E8BAECD9
:1004A600E0DEA3E8BAECDDDE0895D0D0AED0F6DF0C
:1004B600CFDFEB36E1F4CCDF1E2FCADF0E2FC8DF0D
:1004C6003E2FC6DF2E2F113331F4023321F433339E
:1004D60011F4263309F001C0949A123331F405332E
:1004E60021F4373311F4223309F001C0C09AC29ABD
:1004F600C49AD4DFB0D0249608957EDE6E2EE4E250
:10050600E61509F49D9A989B06C0E4E2E61511F0FB
:100516009D9B01C001C004C07DD0A62DB7DE87D04B
:10052600EAE0E61509F49D980895FF92AA93869944
:1005360003C06894F0F865D06DD0ABE6A7DEA8815D
:10054600A13041F4A1E3A2DEA2E3A0DEA3E39EDE96
:10055600A6E39CDE6CD0AAE04ED0F0FC56D02196E5
:10056600FF900895AA935D9BFECFE881ECB9219692
:100576000895BA93AA931A93E981FA813196E98389
:10058600FA833197E4911E2FE03019F0A12FEADFAC
:10059600F3CFAAE0E7DF188123960895EFE1EDBDDA
:1005A600E0E0ECBD0895EFB9E1E1EDB9E3E1EDB9C5
:1005B600E1E1EDB9E3E1EDB9E1E1EDB9E3E1EDB991
:1005C600E1E1EDB9E3E1EDB9E1E1EDB9E3E1EDB981
:1005D600E1E1EDB9E3E1EDB9E1E1EDB9E3E1EDB971
:1005E600E1E1EDB9E3E1EDB9EFB10895E1E1EDB98E
:1005F600E3E1EDB90895B0E01FC0EA93A4EFB1E0DE
:100606001DCE969AA9E3B2E82CCEA9EDB2E829DE72
:1006160096980895C29AA0E0B0E023DEC498A8EBAD
:1006260035DEAAEA33DEADE231DEA6ED2FCEA0E05E
:100636002DDEC298C49A0895109639F086E69EE09B
:100646000197F1F7A8951197C9F708953A932A9358
:100656001A930A9308953B812A8119810881089586
:00000001FF
